 jimage

 Timestamp is e90d689f (reproducible build file hash)

 Preferred load address is 0000000180000000

 Start         Length     Name                   Class
 0001:00000000 00000030H .text$di                CODE
 0001:00000030 00002b80H .text$mn                CODE
 0001:00002bb0 00000036H .text$mn$00             CODE
 0001:00002be6 00000092H .text$x                 CODE
 0002:00000000 00000208H .idata$5                DATA
 0002:00000208 00000038H .00cfg                  DATA
 0002:00000240 00000008H .CRT$XCA                DATA
 0002:00000248 00000010H .CRT$XCU                DATA
 0002:00000258 00000008H .CRT$XCZ                DATA
 0002:00000260 00000008H .CRT$XIA                DATA
 0002:00000268 00000008H .CRT$XIZ                DATA
 0002:00000270 00000008H .CRT$XPA                DATA
 0002:00000278 00000008H .CRT$XPZ                DATA
 0002:00000280 00000008H .CRT$XTA                DATA
 0002:00000288 00000008H .CRT$XTZ                DATA
 0002:00000290 00000000H .gehcont$y              DATA
 0002:00000290 00000000H .gfids$y                DATA
 0002:00000290 00000470H .rdata                  DATA
 0002:00000700 00000000H .rdata$CastGuardVftablesA DATA
 0002:00000700 00000000H .rdata$CastGuardVftablesC DATA
 0002:00000700 00000494H .rdata$r                DATA
 0002:00000b94 00000080H .rdata$voltmd           DATA
 0002:00000c14 0000032cH .rdata$zzzdbg           DATA
 0002:00000f40 00000008H .rtc$IAA                DATA
 0002:00000f48 00000008H .rtc$IZZ                DATA
 0002:00000f50 00000008H .rtc$TAA                DATA
 0002:00000f58 00000008H .rtc$TZZ                DATA
 0002:00000f60 00000318H .xdata                  DATA
 0002:00001278 000000f8H .xdata$x                DATA
 0002:00001370 00000120H .edata                  DATA
 0002:00001490 000000a0H .idata$2                DATA
 0002:00001530 00000018H .idata$3                DATA
 0002:00001548 00000208H .idata$4                DATA
 0002:00001750 0000050aH .idata$6                DATA
 0003:00000000 000000c8H .data                   DATA
 0003:000000c8 00000080H .data$r                 DATA
 0003:00000148 00000118H .data$rs                DATA
 0003:00000260 00000648H .bss                    DATA
 0004:00000000 000003f0H .pdata                  DATA
 0005:00000000 00000060H .rsrc$01                DATA
 0005:00000060 00000340H .rsrc$02                DATA

  Address         Publics by Value              Rva+Base               Lib:Object

 0000:00000000       __AbsoluteZero             0000000000000000     <absolute>
 0000:00000000       ___safe_se_handler_count   0000000000000000     <absolute>
 0000:00000000       ___safe_se_handler_table   0000000000000000     <absolute>
 0000:00000000       __arm64x_extra_rfe_table   0000000000000000     <absolute>
 0000:00000000       __arm64x_extra_rfe_table_size 0000000000000000     <absolute>
 0000:00000000       __arm64x_native_entrypoint 0000000000000000     <absolute>
 0000:00000000       __arm64x_redirection_metadata 0000000000000000     <absolute>
 0000:00000000       __arm64x_redirection_metadata_count 0000000000000000     <absolute>
 0000:00000000       __dynamic_value_reloc_table 0000000000000000     <absolute>
 0000:00000000       __enclave_config           0000000000000000     <absolute>
 0000:00000000       __guard_check_icall_a64n_fptr 0000000000000000     <absolute>
 0000:00000000       __guard_eh_cont_count      0000000000000000     <absolute>
 0000:00000000       __guard_eh_cont_table      0000000000000000     <absolute>
 0000:00000000       __guard_fids_count         0000000000000000     <absolute>
 0000:00000000       __guard_fids_table         0000000000000000     <absolute>
 0000:00000000       __guard_iat_count          0000000000000000     <absolute>
 0000:00000000       __guard_iat_table          0000000000000000     <absolute>
 0000:00000000       __guard_longjmp_count      0000000000000000     <absolute>
 0000:00000000       __guard_longjmp_table      0000000000000000     <absolute>
 0000:00000000       __hybrid_auxiliary_delayload_iat 0000000000000000     <absolute>
 0000:00000000       __hybrid_auxiliary_delayload_iat_copy 0000000000000000     <absolute>
 0000:00000000       __hybrid_auxiliary_iat     0000000000000000     <absolute>
 0000:00000000       __hybrid_auxiliary_iat_copy 0000000000000000     <absolute>
 0000:00000000       __hybrid_code_map          0000000000000000     <absolute>
 0000:00000000       __hybrid_code_map_count    0000000000000000     <absolute>
 0000:00000000       __hybrid_image_info_bitfield 0000000000000000     <absolute>
 0000:00000000       __x64_code_ranges_to_entry_points 0000000000000000     <absolute>
 0000:00000000       __x64_code_ranges_to_entry_points_count 0000000000000000     <absolute>
 0000:00000100       __guard_flags              0000000000000100     <absolute>
 0000:00000000       __ImageBase                0000000180000000     <linker-defined>
 0001:00000030       Java_jdk_internal_jimage_NativeImageBuffer_getNativeMap 0000000180001030 f   NativeImageBuffer.obj
 0001:000000c0       ?get@NativeEndian@@UEAAFF@Z 00000001800010c0 f   endian.obj
 0001:000000c0       ?get@NativeEndian@@UEAAGG@Z 00000001800010c0 f   endian.obj
 0001:000000c4       ?get@NativeEndian@@UEAAHH@Z 00000001800010c4 f   endian.obj
 0001:000000c4       ?get@NativeEndian@@UEAAII@Z 00000001800010c4 f   endian.obj
 0001:000000c8       ?get@NativeEndian@@UEAA_J_J@Z 00000001800010c8 f   endian.obj
 0001:000000c8       ?get@NativeEndian@@UEAA_K_K@Z 00000001800010c8 f   endian.obj
 0001:000000cc       ?set@NativeEndian@@UEAAXAEAFF@Z 00000001800010cc f   endian.obj
 0001:000000cc       ?set@NativeEndian@@UEAAXAEAGG@Z 00000001800010cc f   endian.obj
 0001:000000d4       ?set@NativeEndian@@UEAAXAEAHH@Z 00000001800010d4 f   endian.obj
 0001:000000d4       ?set@NativeEndian@@UEAAXAEAII@Z 00000001800010d4 f   endian.obj
 0001:000000d8       ?set@NativeEndian@@UEAAXAEA_J_J@Z 00000001800010d8 f   endian.obj
 0001:000000d8       ?set@NativeEndian@@UEAAXAEA_K_K@Z 00000001800010d8 f   endian.obj
 0001:000000dc       ?get@SwappingEndian@@UEAAFF@Z 00000001800010dc f   endian.obj
 0001:000000dc       ?get@SwappingEndian@@UEAAGG@Z 00000001800010dc f   endian.obj
 0001:000000e4       ?get@SwappingEndian@@UEAAHH@Z 00000001800010e4 f   endian.obj
 0001:000000e4       ?get@SwappingEndian@@UEAAII@Z 00000001800010e4 f   endian.obj
 0001:000000ec       ?get@SwappingEndian@@UEAA_J_J@Z 00000001800010ec f   endian.obj
 0001:000000ec       ?get@SwappingEndian@@UEAA_K_K@Z 00000001800010ec f   endian.obj
 0001:0000015c       ?set@SwappingEndian@@UEAAXAEAFF@Z 000000018000115c f   endian.obj
 0001:0000015c       ?set@SwappingEndian@@UEAAXAEAGG@Z 000000018000115c f   endian.obj
 0001:00000168       ?set@SwappingEndian@@UEAAXAEAHH@Z 0000000180001168 f   endian.obj
 0001:00000168       ?set@SwappingEndian@@UEAAXAEAII@Z 0000000180001168 f   endian.obj
 0001:00000170       ?set@SwappingEndian@@UEAAXAEA_J_J@Z 0000000180001170 f   endian.obj
 0001:00000170       ?set@SwappingEndian@@UEAAXAEA_K_K@Z 0000000180001170 f   endian.obj
 0001:000001e4       ?get_handler@Endian@@SAPEAV1@_N@Z 00000001800011e4 f   endian.obj
 0001:000001fc       ?get_java@Endian@@SAGPEAE@Z 00000001800011fc f   endian.obj
 0001:0000020c       ?set_java@Endian@@SAXPEAEG@Z 000000018000120c f   endian.obj
 0001:0000021c       ?decompress_int@SharedStringDecompressor@@CAHAEAPEAE@Z 000000018000121c f   imageDecompressor.obj
 0001:000002b4       ?decompress_resource@ImageDecompressor@@SAXPEAE0_KPEBVImageStrings@@PEAVEndian@@@Z 00000001800012b4 f   imageDecompressor.obj
 0001:00000484       ?decompress_resource@SharedStringDecompressor@@UEAAXPEAE0PEAUResourceHeader@@PEBVImageStrings@@@Z 0000000180001484 f   imageDecompressor.obj
 0001:0000079c       ?decompress_resource@ZipDecompressor@@UEAAXPEAE0PEAUResourceHeader@@PEBVImageStrings@@@Z 000000018000179c f   imageDecompressor.obj
 0001:000007cc       ?get_decompressor@ImageDecompressor@@SAPEAV1@PEBD@Z 00000001800017cc f   imageDecompressor.obj
 0001:0000083c       ?image_decompressor_init@ImageDecompressor@@SAXXZ 000000018000183c f   imageDecompressor.obj
 0001:000008e8       __local_stdio_printf_options 00000001800018e8 f i imageDecompressor.obj
 0001:000008f0       printf                     00000001800018f0 f i imageDecompressor.obj
 0001:00000944       ??0ImageFileReader@@AEAA@PEBD_N@Z 0000000180001944 f   imageFile.obj
 0001:000009c0       ??1ImageFileReader@@AEAA@XZ 00000001800019c0 f   imageFile.obj
 0001:000009f8       ?add@ImageFileReaderTable@@QEAAXPEAVImageFileReader@@@Z 00000001800019f8 f   imageFile.obj
 0001:00000a4c       ?clear_data@ImageLocation@@QEAAXXZ 0000000180001a4c f   imageFile.obj
 0001:00000a58       ?close@ImageFileReader@@QEAAXXZ 0000000180001a58 f   imageFile.obj
 0001:00000ab8       ?close@ImageFileReader@@SAXPEAV1@@Z 0000000180001ab8 f   imageFile.obj
 0001:00000b08       ?find@ImageStrings@@SAHPEAVEndian@@PEBDPEAHI@Z 0000000180001b08 f   imageFile.obj
 0001:00000bb0       ?find_image@ImageFileReader@@SAPEAV1@PEBD@Z 0000000180001bb0 f   imageFile.obj
 0001:00000c24       ?find_location@ImageFileReader@@QEBA_NPEBDAEAVImageLocation@@@Z 0000000180001c24 f   imageFile.obj
 0001:00000cac       ?find_location_index@ImageFileReader@@QEBAIPEBDPEA_K@Z 0000000180001cac f   imageFile.obj
 0001:00000d70       ?get_image_module_data@ImageFileReader@@QEAAPEAVImageModuleData@@XZ 0000000180001d70 f   imageFile.obj
 0001:00000d78       ?get_resource@ImageFileReader@@QEBAXAEAVImageLocation@@PEAE@Z 0000000180001d78 f   imageFile.obj
 0001:00000e54       ?get_resource@ImageFileReader@@QEBAXIPEAE@Z 0000000180001e54 f   imageFile.obj
 0001:00000ec0       ?open@ImageFileReader@@QEAA_NXZ 0000000180001ec0 f   imageFile.obj
 0001:00001050       ?open@ImageFileReader@@SAPEAV1@PEBD_N@Z 0000000180002050 f   imageFile.obj
 0001:00001164       ?package_to_module@ImageModuleData@@QEAAPEBDPEBD@Z 0000000180002164 f   imageFile.obj
 0001:000012ec       ?remove@ImageFileReaderTable@@QEAAXPEAVImageFileReader@@@Z 00000001800022ec f   imageFile.obj
 0001:0000134c       ?set_data@ImageLocation@@QEAAXPEAE@Z 000000018000234c f   imageFile.obj
 0001:000013a8       ?verify_location@ImageFileReader@@QEBA_NAEAVImageLocation@@PEBD@Z 00000001800023a8 f   imageFile.obj
 0001:000014d4       JIMAGE_Close               00000001800024d4 f   jimage.obj
 0001:000014dc       JIMAGE_FindResource        00000001800024dc f   jimage.obj
 0001:000015c4       JIMAGE_GetResource         00000001800025c4 f   jimage.obj
 0001:000015dc       JIMAGE_Open                00000001800025dc f   jimage.obj
 0001:000015e8       JIMAGE_PackageToModule     00000001800025e8 f   jimage.obj
 0001:00001608       JIMAGE_ResourceIterator    0000000180002608 f   jimage.obj
 0001:00001744       ??0SimpleCriticalSection@@QEAA@XZ 0000000180002744 f   osSupport_windows.obj
 0001:0000175c       ?close@osSupport@@SAHH@Z   000000018000275c f   osSupport_windows.obj
 0001:00001764       ?enter@SimpleCriticalSection@@AEAAXXZ 0000000180002764 f   osSupport_windows.obj
 0001:0000176c       ?exit@SimpleCriticalSection@@AEAAXXZ 000000018000276c f   osSupport_windows.obj
 0001:00001774       ?map_memory@osSupport@@SAPEAXHPEBD_K1@Z 0000000180002774 f   osSupport_windows.obj
 0001:00001838       ?openReadOnly@osSupport@@SAHPEBD@Z 0000000180002838 f   osSupport_windows.obj
 0001:00001848       ?read@osSupport@@SA_JHPEAD_J1@Z 0000000180002848 f   osSupport_windows.obj
 0001:000018c8       ?size@osSupport@@SA_JPEBD@Z 00000001800028c8 f   osSupport_windows.obj
 0001:00001914       ?unmap_memory@osSupport@@SAHPEAX_K@Z 0000000180002914 f   osSupport_windows.obj
 0001:0000191b       JVM_LoadZipLibrary         000000018000291b f   jvm:jvm.dll
 0001:00001924       ??_Etype_info@@UEAAPEAXI@Z 0000000180002924 f i MSVCRT:std_type_info_static.obj
 0001:00001924       ??_Gtype_info@@UEAAPEAXI@Z 0000000180002924 f i MSVCRT:std_type_info_static.obj
 0001:00001950       ??2@YAPEAX_K@Z             0000000180002950 f   MSVCRT:new_scalar.obj
 0001:0000198c       ??_U@YAPEAX_K@Z            000000018000298c f   MSVCRT:new_array.obj
 0001:00001994       ??3@YAXPEAX_K@Z            0000000180002994 f   MSVCRT:delete_scalar_size.obj
 0001:00001994       ??_V@YAXPEAX@Z             0000000180002994 f   MSVCRT:delete_array.obj
 0001:0000199c       __GSHandlerCheck           000000018000299c f   MSVCRT:gshandler.obj
 0001:000019bc       __GSHandlerCheckCommon     00000001800029bc f   MSVCRT:gshandler.obj
 0001:00001a30       __security_check_cookie    0000000180002a30 f   MSVCRT:amdsecgs.obj
 0001:00001a50       __raise_securityfailure    0000000180002a50 f   MSVCRT:gs_report.obj
 0001:00001a84       __report_gsfailure         0000000180002a84 f   MSVCRT:gs_report.obj
 0001:00001b58       __report_rangecheckfailure 0000000180002b58 f   MSVCRT:gs_report.obj
 0001:00001b6c       __report_securityfailure   0000000180002b6c f   MSVCRT:gs_report.obj
 0001:00001d00       __chkstk                   0000000180002d00 f   MSVCRT:chkstk.obj
 0001:00001d00       _alloca_probe              0000000180002d00 f   MSVCRT:chkstk.obj
 0001:00002060       _DllMainCRTStartup         0000000180003060 f   MSVCRT:dll_dllmain.obj
 0001:000020a0       ??0bad_alloc@std@@QEAA@AEBV01@@Z 00000001800030a0 f i MSVCRT:throw_bad_alloc.obj
 0001:000020dc       ??0bad_alloc@std@@QEAA@XZ  00000001800030dc f i MSVCRT:throw_bad_alloc.obj
 0001:000020fc       ??0bad_array_new_length@std@@QEAA@AEBV01@@Z 00000001800030fc f i MSVCRT:throw_bad_alloc.obj
 0001:00002138       ??0bad_array_new_length@std@@QEAA@XZ 0000000180003138 f i MSVCRT:throw_bad_alloc.obj
 0001:00002158       ??0exception@std@@QEAA@AEBV01@@Z 0000000180003158 f i MSVCRT:throw_bad_alloc.obj
 0001:0000218c       ??1bad_alloc@std@@UEAA@XZ  000000018000318c f i MSVCRT:throw_bad_alloc.obj
 0001:0000218c       ??1bad_array_new_length@std@@UEAA@XZ 000000018000318c f i MSVCRT:throw_bad_alloc.obj
 0001:000021a0       ??_Ebad_alloc@std@@UEAAPEAXI@Z 00000001800031a0 f i MSVCRT:throw_bad_alloc.obj
 0001:000021a0       ??_Ebad_array_new_length@std@@UEAAPEAXI@Z 00000001800031a0 f i MSVCRT:throw_bad_alloc.obj
 0001:000021a0       ??_Eexception@std@@UEAAPEAXI@Z 00000001800031a0 f i MSVCRT:throw_bad_alloc.obj
 0001:000021a0       ??_Gbad_alloc@std@@UEAAPEAXI@Z 00000001800031a0 f i MSVCRT:throw_bad_alloc.obj
 0001:000021a0       ??_Gbad_array_new_length@std@@UEAAPEAXI@Z 00000001800031a0 f i MSVCRT:throw_bad_alloc.obj
 0001:000021a0       ??_Gexception@std@@UEAAPEAXI@Z 00000001800031a0 f i MSVCRT:throw_bad_alloc.obj
 0001:000021e4       ?__scrt_throw_std_bad_alloc@@YAXXZ 00000001800031e4 f   MSVCRT:throw_bad_alloc.obj
 0001:00002204       ?__scrt_throw_std_bad_array_new_length@@YAXXZ 0000000180003204 f   MSVCRT:throw_bad_alloc.obj
 0001:00002224       ?what@exception@std@@UEBAPEBDXZ 0000000180003224 f i MSVCRT:throw_bad_alloc.obj
 0001:00002238       ??3@YAXPEAX@Z              0000000180003238 f   MSVCRT:delete_scalar.obj
 0001:00002240       __security_init_cookie     0000000180003240 f   MSVCRT:gs_support.obj
 0001:000022ec       DllMain                    00000001800032ec f   MSVCRT:dll_dllmain_stub.obj
 0001:00002310       ?__scrt_initialize_type_info@@YAXXZ 0000000180003310 f   MSVCRT:tncleanup.obj
 0001:00002320       ?__scrt_uninitialize_type_info@@YAXXZ 0000000180003320 f   MSVCRT:tncleanup.obj
 0001:0000232c       __local_stdio_scanf_options 000000018000332c f i MSVCRT:default_local_stdio_options.obj
 0001:00002334       __scrt_initialize_default_local_stdio_options 0000000180003334 f   MSVCRT:default_local_stdio_options.obj
 0001:00002350       __scrt_acquire_startup_lock 0000000180003350 f   MSVCRT:utility.obj
 0001:0000238c       __scrt_dllmain_after_initialize_c 000000018000338c f   MSVCRT:utility.obj
 0001:000023c0       __scrt_dllmain_before_initialize_c 00000001800033c0 f   MSVCRT:utility.obj
 0001:000023d8       __scrt_dllmain_crt_thread_attach 00000001800033d8 f   MSVCRT:utility.obj
 0001:00002400       __scrt_dllmain_crt_thread_detach 0000000180003400 f   MSVCRT:utility.obj
 0001:00002418       __scrt_dllmain_exception_filter 0000000180003418 f   MSVCRT:utility.obj
 0001:00002478       __scrt_dllmain_uninitialize_c 0000000180003478 f   MSVCRT:utility.obj
 0001:000024a8       __scrt_dllmain_uninitialize_critical 00000001800034a8 f   MSVCRT:utility.obj
 0001:000024bc       __scrt_initialize_crt      00000001800034bc f   MSVCRT:utility.obj
 0001:000024f8       __scrt_initialize_onexit_tables 00000001800034f8 f   MSVCRT:utility.obj
 0001:00002584       __scrt_is_nonwritable_in_current_image 0000000180003584 f   MSVCRT:utility.obj
 0001:0000261c       __scrt_release_startup_lock 000000018000361c f   MSVCRT:utility.obj
 0001:00002640       __scrt_uninitialize_crt    0000000180003640 f   MSVCRT:utility.obj
 0001:0000266c       __scrt_get_dyn_tls_init_callback 000000018000366c f   MSVCRT:dyn_tls_init.obj
 0001:00002674       __crt_debugger_hook        0000000180003674 f   MSVCRT:utility_desktop.obj
 0001:0000267c       __scrt_fastfail            000000018000367c f   MSVCRT:utility_desktop.obj
 0001:000027c4       _RTC_Initialize            00000001800037c4 f   MSVCRT:initsect.obj
 0001:00002800       _RTC_Terminate             0000000180003800 f   MSVCRT:initsect.obj
 0001:0000283c       _guard_check_icall_nop     000000018000383c f i MSVCRT:guard_support.obj
 0001:00002840       __isa_available_init       0000000180003840 f   MSVCRT:cpu_disp.obj
 0001:00002b0c       _get_startup_argv_mode     0000000180003b0c f   MSVCRT:argv_mode.obj
 0001:00002b14       __scrt_is_ucrt_dll_in_use  0000000180003b14 f   MSVCRT:ucrt_detection.obj
 0001:00002b20       memcpy                     0000000180003b20 f   vcruntime:VCRUNTIME140.dll
 0001:00002b26       memset                     0000000180003b26 f   vcruntime:VCRUNTIME140.dll
 0001:00002b2c       __C_specific_handler       0000000180003b2c f   vcruntime:VCRUNTIME140.dll
 0001:00002b32       __std_exception_copy       0000000180003b32 f   vcruntime:VCRUNTIME140.dll
 0001:00002b38       __std_exception_destroy    0000000180003b38 f   vcruntime:VCRUNTIME140.dll
 0001:00002b3e       _CxxThrowException         0000000180003b3e f   vcruntime:VCRUNTIME140.dll
 0001:00002b44       __std_type_info_destroy_list 0000000180003b44 f   vcruntime:VCRUNTIME140.dll
 0001:00002b4a       strcmp                     0000000180003b4a f   ucrt:api-ms-win-crt-string-l1-1-0.dll
 0001:00002b50       strlen                     0000000180003b50 f   ucrt:api-ms-win-crt-string-l1-1-0.dll
 0001:00002b56       strcat                     0000000180003b56 f   ucrt:api-ms-win-crt-string-l1-1-0.dll
 0001:00002b5c       strcpy                     0000000180003b5c f   ucrt:api-ms-win-crt-string-l1-1-0.dll
 0001:00002b62       _callnewh                  0000000180003b62 f   ucrt:api-ms-win-crt-heap-l1-1-0.dll
 0001:00002b68       malloc                     0000000180003b68 f   ucrt:api-ms-win-crt-heap-l1-1-0.dll
 0001:00002b6e       _initterm                  0000000180003b6e f   ucrt:api-ms-win-crt-runtime-l1-1-0.dll
 0001:00002b74       _initterm_e                0000000180003b74 f   ucrt:api-ms-win-crt-runtime-l1-1-0.dll
 0001:00002b7a       free                       0000000180003b7a f   ucrt:api-ms-win-crt-heap-l1-1-0.dll
 0001:00002b80       _seh_filter_dll            0000000180003b80 f   ucrt:api-ms-win-crt-runtime-l1-1-0.dll
 0001:00002b86       _configure_narrow_argv     0000000180003b86 f   ucrt:api-ms-win-crt-runtime-l1-1-0.dll
 0001:00002b8c       _initialize_narrow_environment 0000000180003b8c f   ucrt:api-ms-win-crt-runtime-l1-1-0.dll
 0001:00002b92       _initialize_onexit_table   0000000180003b92 f   ucrt:api-ms-win-crt-runtime-l1-1-0.dll
 0001:00002b98       _execute_onexit_table      0000000180003b98 f   ucrt:api-ms-win-crt-runtime-l1-1-0.dll
 0001:00002b9e       _cexit                     0000000180003b9e f   ucrt:api-ms-win-crt-runtime-l1-1-0.dll
 0001:00002ba4       __acrt_initialize          0000000180003ba4 f   MSVCRT:ucrt_stubs.obj
 0001:00002ba4       __acrt_thread_attach       0000000180003ba4 f   MSVCRT:ucrt_stubs.obj
 0001:00002ba4       __acrt_thread_detach       0000000180003ba4 f   MSVCRT:ucrt_stubs.obj
 0001:00002ba4       __acrt_uninitialize        0000000180003ba4 f   MSVCRT:ucrt_stubs.obj
 0001:00002ba4       __acrt_uninitialize_critical 0000000180003ba4 f   MSVCRT:ucrt_stubs.obj
 0001:00002ba4       __scrt_stub_for_acrt_initialize 0000000180003ba4 f   MSVCRT:ucrt_stubs.obj
 0001:00002ba4       __scrt_stub_for_acrt_thread_attach 0000000180003ba4 f   MSVCRT:ucrt_stubs.obj
 0001:00002ba4       __scrt_stub_for_acrt_thread_detach 0000000180003ba4 f   MSVCRT:ucrt_stubs.obj
 0001:00002ba4       __scrt_stub_for_acrt_uninitialize 0000000180003ba4 f   MSVCRT:ucrt_stubs.obj
 0001:00002ba4       __scrt_stub_for_acrt_uninitialize_critical 0000000180003ba4 f   MSVCRT:ucrt_stubs.obj
 0001:00002ba4       __vcrt_initialize          0000000180003ba4 f   MSVCRT:ucrt_stubs.obj
 0001:00002ba4       __vcrt_thread_attach       0000000180003ba4 f   MSVCRT:ucrt_stubs.obj
 0001:00002ba4       __vcrt_thread_detach       0000000180003ba4 f   MSVCRT:ucrt_stubs.obj
 0001:00002ba4       __vcrt_uninitialize        0000000180003ba4 f   MSVCRT:ucrt_stubs.obj
 0001:00002ba4       __vcrt_uninitialize_critical 0000000180003ba4 f   MSVCRT:ucrt_stubs.obj
 0001:00002ba8       __scrt_stub_for_is_c_termination_complete 0000000180003ba8 f   MSVCRT:ucrt_stubs.obj
 0001:00002ba8       _is_c_termination_complete 0000000180003ba8 f   MSVCRT:ucrt_stubs.obj
 0001:00002bc0       _guard_dispatch_icall_nop  0000000180003bc0 f   MSVCRT:guard_dispatch.obj
 0001:00002be0       _guard_xfg_dispatch_icall_nop 0000000180003be0 f   MSVCRT:guard_xfg_dispatch.obj
 0002:00000000       __imp_UnhandledExceptionFilter 0000000180004000     kernel32:KERNEL32.dll
 0002:00000008       __imp_GetProcAddress       0000000180004008     kernel32:KERNEL32.dll
 0002:00000010       __imp_CreateFileA          0000000180004010     kernel32:KERNEL32.dll
 0002:00000018       __imp_ReadFile             0000000180004018     kernel32:KERNEL32.dll
 0002:00000020       __imp_CloseHandle          0000000180004020     kernel32:KERNEL32.dll
 0002:00000028       __imp_InitializeCriticalSection 0000000180004028     kernel32:KERNEL32.dll
 0002:00000030       __imp_EnterCriticalSection 0000000180004030     kernel32:KERNEL32.dll
 0002:00000038       __imp_LeaveCriticalSection 0000000180004038     kernel32:KERNEL32.dll
 0002:00000040       __imp_MapViewOfFileEx      0000000180004040     kernel32:KERNEL32.dll
 0002:00000048       __imp_UnmapViewOfFile      0000000180004048     kernel32:KERNEL32.dll
 0002:00000050       __imp_CreateFileMappingA   0000000180004050     kernel32:KERNEL32.dll
 0002:00000058       __imp_RtlCaptureContext    0000000180004058     kernel32:KERNEL32.dll
 0002:00000060       __imp_RtlLookupFunctionEntry 0000000180004060     kernel32:KERNEL32.dll
 0002:00000068       __imp_RtlVirtualUnwind     0000000180004068     kernel32:KERNEL32.dll
 0002:00000070       __imp_IsDebuggerPresent    0000000180004070     kernel32:KERNEL32.dll
 0002:00000078       __imp_SetUnhandledExceptionFilter 0000000180004078     kernel32:KERNEL32.dll
 0002:00000080       __imp_GetCurrentProcess    0000000180004080     kernel32:KERNEL32.dll
 0002:00000088       __imp_TerminateProcess     0000000180004088     kernel32:KERNEL32.dll
 0002:00000090       __imp_IsProcessorFeaturePresent 0000000180004090     kernel32:KERNEL32.dll
 0002:00000098       __imp_QueryPerformanceCounter 0000000180004098     kernel32:KERNEL32.dll
 0002:000000a0       __imp_GetCurrentProcessId  00000001800040a0     kernel32:KERNEL32.dll
 0002:000000a8       __imp_GetCurrentThreadId   00000001800040a8     kernel32:KERNEL32.dll
 0002:000000b0       __imp_GetSystemTimeAsFileTime 00000001800040b0     kernel32:KERNEL32.dll
 0002:000000b8       __imp_DisableThreadLibraryCalls 00000001800040b8     kernel32:KERNEL32.dll
 0002:000000c0       __imp_InitializeSListHead  00000001800040c0     kernel32:KERNEL32.dll
 0002:000000c8       \177KERNEL32_NULL_THUNK_DATA 00000001800040c8     kernel32:KERNEL32.dll
 0002:000000d0       __imp___std_type_info_destroy_list 00000001800040d0     vcruntime:VCRUNTIME140.dll
 0002:000000d8       __imp_memcpy               00000001800040d8     vcruntime:VCRUNTIME140.dll
 0002:000000e0       __imp_memset               00000001800040e0     vcruntime:VCRUNTIME140.dll
 0002:000000e8       __imp___C_specific_handler 00000001800040e8     vcruntime:VCRUNTIME140.dll
 0002:000000f0       __imp___std_exception_copy 00000001800040f0     vcruntime:VCRUNTIME140.dll
 0002:000000f8       __imp___std_exception_destroy 00000001800040f8     vcruntime:VCRUNTIME140.dll
 0002:00000100       __imp__CxxThrowException   0000000180004100     vcruntime:VCRUNTIME140.dll
 0002:00000108       \177VCRUNTIME140_NULL_THUNK_DATA 0000000180004108     vcruntime:VCRUNTIME140.dll
 0002:00000110       __imp__stat64i32           0000000180004110     ucrt:api-ms-win-crt-filesystem-l1-1-0.dll
 0002:00000118       \177api-ms-win-crt-filesystem-l1-1-0_NULL_THUNK_DATA 0000000180004118     ucrt:api-ms-win-crt-filesystem-l1-1-0.dll
 0002:00000120       __imp__callnewh            0000000180004120     ucrt:api-ms-win-crt-heap-l1-1-0.dll
 0002:00000128       __imp_malloc               0000000180004128     ucrt:api-ms-win-crt-heap-l1-1-0.dll
 0002:00000130       __imp_realloc              0000000180004130     ucrt:api-ms-win-crt-heap-l1-1-0.dll
 0002:00000138       __imp_calloc               0000000180004138     ucrt:api-ms-win-crt-heap-l1-1-0.dll
 0002:00000140       __imp_free                 0000000180004140     ucrt:api-ms-win-crt-heap-l1-1-0.dll
 0002:00000148       \177api-ms-win-crt-heap-l1-1-0_NULL_THUNK_DATA 0000000180004148     ucrt:api-ms-win-crt-heap-l1-1-0.dll
 0002:00000150       __imp__initialize_narrow_environment 0000000180004150     ucrt:api-ms-win-crt-runtime-l1-1-0.dll
 0002:00000158       __imp__cexit               0000000180004158     ucrt:api-ms-win-crt-runtime-l1-1-0.dll
 0002:00000160       __imp__initialize_onexit_table 0000000180004160     ucrt:api-ms-win-crt-runtime-l1-1-0.dll
 0002:00000168       __imp__execute_onexit_table 0000000180004168     ucrt:api-ms-win-crt-runtime-l1-1-0.dll
 0002:00000170       __imp__initterm            0000000180004170     ucrt:api-ms-win-crt-runtime-l1-1-0.dll
 0002:00000178       __imp__initterm_e          0000000180004178     ucrt:api-ms-win-crt-runtime-l1-1-0.dll
 0002:00000180       __imp__seh_filter_dll      0000000180004180     ucrt:api-ms-win-crt-runtime-l1-1-0.dll
 0002:00000188       __imp__configure_narrow_argv 0000000180004188     ucrt:api-ms-win-crt-runtime-l1-1-0.dll
 0002:00000190       \177api-ms-win-crt-runtime-l1-1-0_NULL_THUNK_DATA 0000000180004190     ucrt:api-ms-win-crt-runtime-l1-1-0.dll
 0002:00000198       __imp__get_osfhandle       0000000180004198     ucrt:api-ms-win-crt-stdio-l1-1-0.dll
 0002:000001a0       __imp___acrt_iob_func      00000001800041a0     ucrt:api-ms-win-crt-stdio-l1-1-0.dll
 0002:000001a8       __imp__open                00000001800041a8     ucrt:api-ms-win-crt-stdio-l1-1-0.dll
 0002:000001a8       __imp_open                 00000001800041a8     ucrt:api-ms-win-crt-stdio-l1-1-0.dll
 0002:000001b0       __imp__close               00000001800041b0     ucrt:api-ms-win-crt-stdio-l1-1-0.dll
 0002:000001b0       __imp_close                00000001800041b0     ucrt:api-ms-win-crt-stdio-l1-1-0.dll
 0002:000001b8       __imp___stdio_common_vfprintf 00000001800041b8     ucrt:api-ms-win-crt-stdio-l1-1-0.dll
 0002:000001c0       \177api-ms-win-crt-stdio-l1-1-0_NULL_THUNK_DATA 00000001800041c0     ucrt:api-ms-win-crt-stdio-l1-1-0.dll
 0002:000001c8       __imp_strlen               00000001800041c8     ucrt:api-ms-win-crt-string-l1-1-0.dll
 0002:000001d0       __imp_strcat               00000001800041d0     ucrt:api-ms-win-crt-string-l1-1-0.dll
 0002:000001d8       __imp_strcpy               00000001800041d8     ucrt:api-ms-win-crt-string-l1-1-0.dll
 0002:000001e0       __imp_strcmp               00000001800041e0     ucrt:api-ms-win-crt-string-l1-1-0.dll
 0002:000001e8       __imp_strncpy              00000001800041e8     ucrt:api-ms-win-crt-string-l1-1-0.dll
 0002:000001f0       \177api-ms-win-crt-string-l1-1-0_NULL_THUNK_DATA 00000001800041f0     ucrt:api-ms-win-crt-string-l1-1-0.dll
 0002:000001f8       __imp_JVM_LoadZipLibrary   00000001800041f8     jvm:jvm.dll
 0002:00000200       \177jvm_NULL_THUNK_DATA    0000000180004200     jvm:jvm.dll
 0002:00000208       __guard_check_icall_fptr   0000000180004208     MSVCRT:guard_support.obj
 0002:00000210       __guard_xfg_check_icall_fptr 0000000180004210     MSVCRT:guard_support.obj
 0002:00000218       __guard_dispatch_icall_fptr 0000000180004218     MSVCRT:guard_support.obj
 0002:00000220       __guard_xfg_dispatch_icall_fptr 0000000180004220     MSVCRT:guard_support.obj
 0002:00000228       __guard_xfg_table_dispatch_icall_fptr 0000000180004228     MSVCRT:guard_support.obj
 0002:00000230       __castguard_check_failure_os_handled_fptr 0000000180004230     MSVCRT:guard_support.obj
 0002:00000238       __guard_memcpy_fptr        0000000180004238     vcruntime:softmemtag.obj
 0002:00000240       __xc_a                     0000000180004240     MSVCRT:initializers.obj
 0002:00000258       __xc_z                     0000000180004258     MSVCRT:initializers.obj
 0002:00000260       __xi_a                     0000000180004260     MSVCRT:initializers.obj
 0002:00000268       __xi_z                     0000000180004268     MSVCRT:initializers.obj
 0002:00000270       __xp_a                     0000000180004270     MSVCRT:initializers.obj
 0002:00000278       __xp_z                     0000000180004278     MSVCRT:initializers.obj
 0002:00000280       __xt_a                     0000000180004280     MSVCRT:initializers.obj
 0002:00000288       __xt_z                     0000000180004288     MSVCRT:initializers.obj
 0002:00000298       ??_7NativeEndian@@6B@      0000000180004298     endian.obj
 0002:00000300       ??_7SwappingEndian@@6B@    0000000180004300     endian.obj
 0002:00000360       ?sizes@SharedStringDecompressor@@0QBEB 0000000180004360     imageDecompressor.obj
 0002:00000380       ??_7ZipDecompressor@@6B@   0000000180004380     imageDecompressor.obj
 0002:00000390       ??_7SharedStringDecompressor@@6B@ 0000000180004390     imageDecompressor.obj
 0002:00000398       ??_C@_0BB@FGJGIFHO@ZIP_InflateFully@ 0000000180004398     imageDecompressor.obj
 0002:000003ac       ??_C@_03LCAAOJEC@zip@      00000001800043ac     imageDecompressor.obj
 0002:000003b0       ??_C@_0L@OENLBBHC@compact?9cp@ 00000001800043b0     imageDecompressor.obj
 0002:000003c0       ??_C@_0CK@CHFPEALO@Failure?0?5expecting?5?$CFllu?5but?5get@ 00000001800043c0     imageDecompressor.obj
 0002:000003f0       ??_C@_0L@ELHBAEMN@?1packages?1@ 00000001800043f0     imageFile.obj
 0002:00000400       ??_C@_07DFGEOAEG@modules@  0000000180004400     jimage.obj
 0002:00000408       ??_C@_08GFNEJDPJ@packages@ 0000000180004408     jimage.obj
 0002:00000414       ??_C@_01LAKCGALK@9@        0000000180004414     jimage.obj
 0002:00000420       ??_7type_info@@6B@         0000000180004420     MSVCRT:std_type_info_static.obj
 0002:00000438       _pDefaultRawDllMain        0000000180004438     MSVCRT:dll_dllmain.obj
 0002:00000438       _pRawDllMain               0000000180004438     MSVCRT:dll_dllmain.obj
 0002:00000448       ??_7exception@std@@6B@     0000000180004448     MSVCRT:throw_bad_alloc.obj
 0002:00000458       ??_C@_0BC@EOODALEL@Unknown?5exception@ 0000000180004458     MSVCRT:throw_bad_alloc.obj
 0002:00000478       ??_7bad_alloc@std@@6B@     0000000180004478     MSVCRT:throw_bad_alloc.obj
 0002:00000488       ??_C@_0P@GHFPNOJB@bad?5allocation@ 0000000180004488     MSVCRT:throw_bad_alloc.obj
 0002:000004a0       ??_7bad_array_new_length@std@@6B@ 00000001800044a0     MSVCRT:throw_bad_alloc.obj
 0002:000004b0       ??_C@_0BF@KINCDENJ@bad?5array?5new?5length@ 00000001800044b0     MSVCRT:throw_bad_alloc.obj
 0002:000004d0       __xmm@ffffffffffffffffffffffffffffffff 00000001800044d0     MSVCRT:utility.obj
 0002:000004e0       _load_config_used          00000001800044e0     MSVCRT:loadcfg.obj
 0002:00000700       ??_R3Endian@@8             0000000180004700     endian.obj
 0002:00000718       ??_R2Endian@@8             0000000180004718     endian.obj
 0002:00000728       ??_R1A@?0A@EA@Endian@@8    0000000180004728     endian.obj
 0002:00000750       ??_R4NativeEndian@@6B@     0000000180004750     endian.obj
 0002:00000778       ??_R3NativeEndian@@8       0000000180004778     endian.obj
 0002:00000790       ??_R2NativeEndian@@8       0000000180004790     endian.obj
 0002:000007a8       ??_R1A@?0A@EA@NativeEndian@@8 00000001800047a8     endian.obj
 0002:000007d0       ??_R4SwappingEndian@@6B@   00000001800047d0     endian.obj
 0002:000007f8       ??_R3SwappingEndian@@8     00000001800047f8     endian.obj
 0002:00000810       ??_R2SwappingEndian@@8     0000000180004810     endian.obj
 0002:00000828       ??_R1A@?0A@EA@SwappingEndian@@8 0000000180004828     endian.obj
 0002:00000850       ??_R3ImageDecompressor@@8  0000000180004850     imageDecompressor.obj
 0002:00000868       ??_R2ImageDecompressor@@8  0000000180004868     imageDecompressor.obj
 0002:00000878       ??_R1A@?0A@EA@ImageDecompressor@@8 0000000180004878     imageDecompressor.obj
 0002:000008a0       ??_R4ZipDecompressor@@6B@  00000001800048a0     imageDecompressor.obj
 0002:000008c8       ??_R3ZipDecompressor@@8    00000001800048c8     imageDecompressor.obj
 0002:000008e0       ??_R2ZipDecompressor@@8    00000001800048e0     imageDecompressor.obj
 0002:000008f8       ??_R1A@?0A@EA@ZipDecompressor@@8 00000001800048f8     imageDecompressor.obj
 0002:00000920       ??_R4SharedStringDecompressor@@6B@ 0000000180004920     imageDecompressor.obj
 0002:00000948       ??_R3SharedStringDecompressor@@8 0000000180004948     imageDecompressor.obj
 0002:00000960       ??_R2SharedStringDecompressor@@8 0000000180004960     imageDecompressor.obj
 0002:00000978       ??_R1A@?0A@EA@SharedStringDecompressor@@8 0000000180004978     imageDecompressor.obj
 0002:000009a0       ??_R4type_info@@6B@        00000001800049a0     MSVCRT:std_type_info_static.obj
 0002:000009c8       ??_R3type_info@@8          00000001800049c8     MSVCRT:std_type_info_static.obj
 0002:000009e0       ??_R2type_info@@8          00000001800049e0     MSVCRT:std_type_info_static.obj
 0002:000009f0       ??_R1A@?0A@EA@type_info@@8 00000001800049f0     MSVCRT:std_type_info_static.obj
 0002:00000a18       ??_R4exception@std@@6B@    0000000180004a18     MSVCRT:throw_bad_alloc.obj
 0002:00000a40       ??_R3exception@std@@8      0000000180004a40     MSVCRT:throw_bad_alloc.obj
 0002:00000a58       ??_R2exception@std@@8      0000000180004a58     MSVCRT:throw_bad_alloc.obj
 0002:00000a68       ??_R1A@?0A@EA@exception@std@@8 0000000180004a68     MSVCRT:throw_bad_alloc.obj
 0002:00000a90       ??_R4bad_array_new_length@std@@6B@ 0000000180004a90     MSVCRT:throw_bad_alloc.obj
 0002:00000ab8       ??_R3bad_array_new_length@std@@8 0000000180004ab8     MSVCRT:throw_bad_alloc.obj
 0002:00000ad0       ??_R2bad_array_new_length@std@@8 0000000180004ad0     MSVCRT:throw_bad_alloc.obj
 0002:00000af0       ??_R1A@?0A@EA@bad_array_new_length@std@@8 0000000180004af0     MSVCRT:throw_bad_alloc.obj
 0002:00000b18       ??_R1A@?0A@EA@bad_alloc@std@@8 0000000180004b18     MSVCRT:throw_bad_alloc.obj
 0002:00000b40       ??_R3bad_alloc@std@@8      0000000180004b40     MSVCRT:throw_bad_alloc.obj
 0002:00000b58       ??_R2bad_alloc@std@@8      0000000180004b58     MSVCRT:throw_bad_alloc.obj
 0002:00000b70       ??_R4bad_alloc@std@@6B@    0000000180004b70     MSVCRT:throw_bad_alloc.obj
 0002:00000b94       __volatile_metadata        0000000180004b94     <linker-defined>
 0002:00000f40       __rtc_iaa                  0000000180004f40     MSVCRT:initsect.obj
 0002:00000f48       __rtc_izz                  0000000180004f48     MSVCRT:initsect.obj
 0002:00000f50       __rtc_taa                  0000000180004f50     MSVCRT:initsect.obj
 0002:00000f58       __rtc_tzz                  0000000180004f58     MSVCRT:initsect.obj
 0002:00001278       _TI2?AVbad_alloc@std@@     0000000180005278     MSVCRT:throw_bad_alloc.obj
 0002:00001298       _CTA2?AVbad_alloc@std@@    0000000180005298     MSVCRT:throw_bad_alloc.obj
 0002:000012b0       _CT??_R0?AVbad_alloc@std@@@8??0bad_alloc@std@@QEAA@AEBV01@@Z24 00000001800052b0     MSVCRT:throw_bad_alloc.obj
 0002:000012d8       _CT??_R0?AVexception@std@@@8??0exception@std@@QEAA@AEBV01@@Z24 00000001800052d8     MSVCRT:throw_bad_alloc.obj
 0002:00001300       _TI3?AVbad_array_new_length@std@@ 0000000180005300     MSVCRT:throw_bad_alloc.obj
 0002:00001320       _CTA3?AVbad_array_new_length@std@@ 0000000180005320     MSVCRT:throw_bad_alloc.obj
 0002:00001340       _CT??_R0?AVbad_array_new_length@std@@@8??0bad_array_new_length@std@@QEAA@AEBV01@@Z24 0000000180005340     MSVCRT:throw_bad_alloc.obj
 0002:00001490       __IMPORT_DESCRIPTOR_jvm    0000000180005490     jvm:jvm.dll
 0002:000014a4       __IMPORT_DESCRIPTOR_KERNEL32 00000001800054a4     kernel32:KERNEL32.dll
 0002:000014b8       __IMPORT_DESCRIPTOR_VCRUNTIME140 00000001800054b8     vcruntime:VCRUNTIME140.dll
 0002:000014cc       __IMPORT_DESCRIPTOR_api-ms-win-crt-stdio-l1-1-0 00000001800054cc     ucrt:api-ms-win-crt-stdio-l1-1-0.dll
 0002:000014e0       __IMPORT_DESCRIPTOR_api-ms-win-crt-string-l1-1-0 00000001800054e0     ucrt:api-ms-win-crt-string-l1-1-0.dll
 0002:000014f4       __IMPORT_DESCRIPTOR_api-ms-win-crt-heap-l1-1-0 00000001800054f4     ucrt:api-ms-win-crt-heap-l1-1-0.dll
 0002:00001508       __IMPORT_DESCRIPTOR_api-ms-win-crt-filesystem-l1-1-0 0000000180005508     ucrt:api-ms-win-crt-filesystem-l1-1-0.dll
 0002:0000151c       __IMPORT_DESCRIPTOR_api-ms-win-crt-runtime-l1-1-0 000000018000551c     ucrt:api-ms-win-crt-runtime-l1-1-0.dll
 0002:00001530       __NULL_IMPORT_DESCRIPTOR   0000000180005530     jvm:jvm.dll
 0003:00000000       ?_native@NativeEndian@@0V1@A 0000000180006000     endian.obj
 0003:00000008       ?_swapping@SwappingEndian@@0V1@A 0000000180006008     endian.obj
 0003:00000010       ?memory_map_image@ImageFileReader@@0_NA 0000000180006010     imageFile.obj
 0003:00000018       ?_reader_table@ImageFileReader@@0VImageFileReaderTable@@A 0000000180006018     imageFile.obj
 0003:00000040       __security_cookie          0000000180006040     MSVCRT:gs_cookie.obj
 0003:00000080       __security_cookie_complement 0000000180006080     MSVCRT:gs_cookie.obj
 0003:00000090       __scrt_native_dllmain_reason 0000000180006090     MSVCRT:utility.obj
 0003:00000098       __isa_inverted             0000000180006098     MSVCRT:cpu_disp.obj
 0003:000000a0       __isa_available            00000001800060a0     MSVCRT:cpu_disp.obj
 0003:000000a4       __isa_enabled              00000001800060a4     MSVCRT:cpu_disp.obj
 0003:000000a8       __memset_fast_string_threshold 00000001800060a8     MSVCRT:cpu_disp.obj
 0003:000000b0       __memset_nt_threshold      00000001800060b0     MSVCRT:cpu_disp.obj
 0003:000000c0       __scrt_ucrt_dll_is_in_use  00000001800060c0     MSVCRT:ucrt_stubs.obj
 0003:000000c8       ??_R0?AVbad_alloc@std@@@8  00000001800060c8     MSVCRT:throw_bad_alloc.obj
 0003:000000f0       ??_R0?AVexception@std@@@8  00000001800060f0     MSVCRT:throw_bad_alloc.obj
 0003:00000118       ??_R0?AVbad_array_new_length@std@@@8 0000000180006118     MSVCRT:throw_bad_alloc.obj
 0003:00000148       ??_R0?AVEndian@@@8         0000000180006148     endian.obj
 0003:00000168       ??_R0?AVNativeEndian@@@8   0000000180006168     endian.obj
 0003:00000190       ??_R0?AVSwappingEndian@@@8 0000000180006190     endian.obj
 0003:000001b8       ??_R0?AVImageDecompressor@@@8 00000001800061b8     imageDecompressor.obj
 0003:000001e0       ??_R0?AVZipDecompressor@@@8 00000001800061e0     imageDecompressor.obj
 0003:00000208       ??_R0?AVSharedStringDecompressor@@@8 0000000180006208     imageDecompressor.obj
 0003:00000238       ??_R0?AVtype_info@@@8      0000000180006238     MSVCRT:std_type_info_static.obj
 0003:00000260       ?_decompressors@ImageDecompressor@@0PEAPEAV1@EA 0000000180006260     imageDecompressor.obj
 0003:00000268       ?_decompressors_num@ImageDecompressor@@0HA 0000000180006268     imageDecompressor.obj
 0003:00000278       ?_OptionsStorage@?1??__local_stdio_printf_options@@9@4_KA 0000000180006278     imageDecompressor.obj
 0003:00000280       ?_reader_table_lock@@3VSimpleCriticalSection@@A 0000000180006280     imageFile.obj
 0003:00000830       ?__type_info_root_node@@3U__type_info_node@@A 0000000180006830     MSVCRT:tncleanup.obj
 0003:00000840       ?_OptionsStorage@?1??__local_stdio_scanf_options@@9@4_KA 0000000180006840     MSVCRT:default_local_stdio_options.obj
 0003:00000848       __scrt_current_native_startup_state 0000000180006848     MSVCRT:utility.obj
 0003:00000850       __scrt_native_startup_lock 0000000180006850     MSVCRT:utility.obj
 0003:00000890       __scrt_debugger_hook_flag  0000000180006890     MSVCRT:utility_desktop.obj
 0003:00000894       __avx10_version            0000000180006894     MSVCRT:cpu_disp.obj
 0003:00000898       __favor                    0000000180006898     MSVCRT:cpu_disp.obj
 0003:000008a0       __dyn_tls_init_callback    00000001800068a0     <common>

 entry point at        0001:00002060

 Static symbols

 0000:ffff6000       .debug$S                   0000000180000000     jimage.exp
 0000:ffff6000       .debug$S                   0000000180000000     vcruntime:VCRUNTIME140.dll
 0000:ffff6000       .debug$S                   0000000180000000     vcruntime:VCRUNTIME140.dll
 0000:ffff6000       .debug$S                   0000000180000000     vcruntime:VCRUNTIME140.dll
 0000:ffff6000       .debug$S                   0000000180000000     vcruntime:VCRUNTIME140.dll
 0000:ffff6000       .debug$S                   0000000180000000     vcruntime:VCRUNTIME140.dll
 0000:ffff6000       .debug$S                   0000000180000000     vcruntime:VCRUNTIME140.dll
 0000:ffff6000       .debug$S                   0000000180000000     vcruntime:VCRUNTIME140.dll
 0000:ffff6000       .debug$S                   0000000180000000     vcruntime:VCRUNTIME140.dll
 0000:ffff6000       .debug$S                   0000000180000000     vcruntime:VCRUNTIME140.dll
 0000:ffff6000       .debug$S                   0000000180000000     vcruntime:VCRUNTIME140.dll
 0000:ffff6000       .debug$S                   0000000180000000     ucrt:api-ms-win-crt-filesystem-l1-1-0.dll
 0000:ffff6000       .debug$S                   0000000180000000     ucrt:api-ms-win-crt-heap-l1-1-0.dll
 0000:ffff6000       .debug$S                   0000000180000000     ucrt:api-ms-win-crt-heap-l1-1-0.dll
 0000:ffff6000       .debug$S                   0000000180000000     ucrt:api-ms-win-crt-heap-l1-1-0.dll
 0000:ffff6000       .debug$S                   0000000180000000     ucrt:api-ms-win-crt-heap-l1-1-0.dll
 0000:ffff6000       .debug$S                   0000000180000000     ucrt:api-ms-win-crt-heap-l1-1-0.dll
 0000:ffff6000       .debug$S                   0000000180000000     ucrt:api-ms-win-crt-runtime-l1-1-0.dll
 0000:ffff6000       .debug$S                   0000000180000000     ucrt:api-ms-win-crt-runtime-l1-1-0.dll
 0000:ffff6000       .debug$S                   0000000180000000     ucrt:api-ms-win-crt-runtime-l1-1-0.dll
 0000:ffff6000       .debug$S                   0000000180000000     ucrt:api-ms-win-crt-runtime-l1-1-0.dll
 0000:ffff6000       .debug$S                   0000000180000000     ucrt:api-ms-win-crt-runtime-l1-1-0.dll
 0000:ffff6000       .debug$S                   0000000180000000     ucrt:api-ms-win-crt-runtime-l1-1-0.dll
 0000:ffff6000       .debug$S                   0000000180000000     ucrt:api-ms-win-crt-runtime-l1-1-0.dll
 0000:ffff6000       .debug$S                   0000000180000000     ucrt:api-ms-win-crt-runtime-l1-1-0.dll
 0000:ffff6000       .debug$S                   0000000180000000     ucrt:api-ms-win-crt-runtime-l1-1-0.dll
 0000:ffff6000       .debug$S                   0000000180000000     ucrt:api-ms-win-crt-runtime-l1-1-0.dll
 0000:ffff6000       .debug$S                   0000000180000000     ucrt:api-ms-win-crt-runtime-l1-1-0.dll
 0000:ffff6000       .debug$S                   0000000180000000     ucrt:api-ms-win-crt-runtime-l1-1-0.dll
 0000:ffff6000       .debug$S                   0000000180000000     ucrt:api-ms-win-crt-stdio-l1-1-0.dll
 0000:ffff6000       .debug$S                   0000000180000000     ucrt:api-ms-win-crt-stdio-l1-1-0.dll
 0000:ffff6000       .debug$S                   0000000180000000     ucrt:api-ms-win-crt-stdio-l1-1-0.dll
 0000:ffff6000       .debug$S                   0000000180000000     ucrt:api-ms-win-crt-stdio-l1-1-0.dll
 0000:ffff6000       .debug$S                   0000000180000000     ucrt:api-ms-win-crt-stdio-l1-1-0.dll
 0000:ffff6000       .debug$S                   0000000180000000     ucrt:api-ms-win-crt-string-l1-1-0.dll
 0000:ffff6000       .debug$S                   0000000180000000     ucrt:api-ms-win-crt-string-l1-1-0.dll
 0000:ffff6000       .debug$S                   0000000180000000     ucrt:api-ms-win-crt-string-l1-1-0.dll
 0000:ffff6000       .debug$S                   0000000180000000     ucrt:api-ms-win-crt-string-l1-1-0.dll
 0000:ffff6000       .debug$S                   0000000180000000     ucrt:api-ms-win-crt-string-l1-1-0.dll
 0000:ffff6000       .debug$S                   0000000180000000     kernel32:KERNEL32.dll
 0000:ffff6000       .debug$S                   0000000180000000     kernel32:KERNEL32.dll
 0000:ffff6000       .debug$S                   0000000180000000     kernel32:KERNEL32.dll
 0000:ffff6000       .debug$S                   0000000180000000     kernel32:KERNEL32.dll
 0000:ffff6000       .debug$S                   0000000180000000     kernel32:KERNEL32.dll
 0000:ffff6000       .debug$S                   0000000180000000     kernel32:KERNEL32.dll
 0000:ffff6000       .debug$S                   0000000180000000     kernel32:KERNEL32.dll
 0000:ffff6000       .debug$S                   0000000180000000     kernel32:KERNEL32.dll
 0000:ffff6000       .debug$S                   0000000180000000     kernel32:KERNEL32.dll
 0000:ffff6000       .debug$S                   0000000180000000     kernel32:KERNEL32.dll
 0000:ffff6000       .debug$S                   0000000180000000     kernel32:KERNEL32.dll
 0000:ffff6000       .debug$S                   0000000180000000     kernel32:KERNEL32.dll
 0000:ffff6000       .debug$S                   0000000180000000     kernel32:KERNEL32.dll
 0000:ffff6000       .debug$S                   0000000180000000     kernel32:KERNEL32.dll
 0000:ffff6000       .debug$S                   0000000180000000     kernel32:KERNEL32.dll
 0000:ffff6000       .debug$S                   0000000180000000     kernel32:KERNEL32.dll
 0000:ffff6000       .debug$S                   0000000180000000     kernel32:KERNEL32.dll
 0000:ffff6000       .debug$S                   0000000180000000     kernel32:KERNEL32.dll
 0000:ffff6000       .debug$S                   0000000180000000     kernel32:KERNEL32.dll
 0000:ffff6000       .debug$S                   0000000180000000     kernel32:KERNEL32.dll
 0000:ffff6000       .debug$S                   0000000180000000     kernel32:KERNEL32.dll
 0000:ffff6000       .debug$S                   0000000180000000     kernel32:KERNEL32.dll
 0000:ffff6000       .debug$S                   0000000180000000     kernel32:KERNEL32.dll
 0000:ffff6000       .debug$S                   0000000180000000     kernel32:KERNEL32.dll
 0000:ffff6000       .debug$S                   0000000180000000     kernel32:KERNEL32.dll
 0000:ffff6000       .debug$S                   0000000180000000     kernel32:KERNEL32.dll
 0000:ffff6000       .debug$S                   0000000180000000     kernel32:KERNEL32.dll
 0000:ffff6000       .debug$S                   0000000180000000     jvm:jvm.dll
 0001:00000000       ??__E?_reader_table@ImageFileReader@@0VImageFileReaderTable@@A@@YAXXZ 0000000180001000 f   imageFile.obj
 0001:00000020       ??__E_reader_table_lock@@YAXXZ 0000000180001020 f   imageFile.obj
 0001:00001a20       $$000000                   0000000180002a20     MSVCRT:amdsecgs.obj
 0001:00001c0c       capture_current_context    0000000180002c0c f   MSVCRT:gs_report.obj
 0001:00001c7c       capture_previous_context   0000000180002c7c f   MSVCRT:gs_report.obj
 0001:00001cf0       $$000000                   0000000180002cf0     MSVCRT:chkstk.obj
 0001:00001d50       ?dllmain_crt_dispatch@@YAHQEAUHINSTANCE__@@KQEAX@Z 0000000180002d50 f   MSVCRT:dll_dllmain.obj
 0001:00001da0       ?dllmain_crt_process_attach@@YAHQEAUHINSTANCE__@@QEAX@Z 0000000180002da0 f   MSVCRT:dll_dllmain.obj
 0001:00001eb8       ?dllmain_crt_process_detach@@YAH_N@Z 0000000180002eb8 f   MSVCRT:dll_dllmain.obj
 0001:00001f38       ?dllmain_dispatch@@YAHQEAUHINSTANCE__@@KQEAX@Z 0000000180002f38 f   MSVCRT:dll_dllmain.obj
 0001:00002bb0       $$000000                   0000000180003bb0     MSVCRT:guard_dispatch.obj
 0001:00002bd0       $$000000                   0000000180003bd0     MSVCRT:guard_xfg_dispatch.obj
 0001:00002be6       ?fin$0@?0??dllmain_crt_process_attach@@YAHQEAUHINSTANCE__@@QEAX@Z@4HA 0000000180003be6 f   MSVCRT:dll_dllmain.obj
 0001:00002bfd       ?fin$0@?0??dllmain_crt_process_detach@@YAH_N@Z@4HA 0000000180003bfd f   MSVCRT:dll_dllmain.obj
 0001:00002c16       ?fin$1@?0??dllmain_crt_process_detach@@YAH_N@Z@4HA 0000000180003c16 f   MSVCRT:dll_dllmain.obj
 0001:00002c2a       ?filt$0@?0??dllmain_dispatch@@YAHQEAUHINSTANCE__@@KQEAX@Z@4HA 0000000180003c2a f   MSVCRT:dll_dllmain.obj
 0001:00002c60       __scrt_is_nonwritable_in_current_image$filt$0 0000000180003c60 f   MSVCRT:utility.obj
 0002:00000248       ??_reader_table$initializer$@ImageFileReader@@0P6AXXZEA@@3P6AXXZEA 0000000180004248     imageFile.obj
 0002:00000250       ?_reader_table_lock$initializer$@@3P6AXXZEA 0000000180004250     imageFile.obj
 0002:00000428       GS_ExceptionPointers       0000000180004428     MSVCRT:gs_report.obj
 0002:00000f60       $unwind$Java_jdk_internal_jimage_NativeImageBuffer_getNativeMap 0000000180004f60     NativeImageBuffer.obj
 0002:00000f60       $unwind$??0ImageFileReader@@AEAA@PEBD_N@Z 0000000180004f60     imageFile.obj
 0002:00000f74       $unwind$printf             0000000180004f74     imageDecompressor.obj
 0002:00000f80       $unwind$?image_decompressor_init@ImageDecompressor@@SAXXZ 0000000180004f80     imageDecompressor.obj
 0002:00000f80       $unwind$??1ImageFileReader@@AEAA@XZ 0000000180004f80     imageFile.obj
 0002:00000f80       $unwind$?close@ImageFileReader@@QEAAXXZ 0000000180004f80     imageFile.obj
 0002:00000f80       $unwind$?close@ImageFileReader@@SAXPEAV1@@Z 0000000180004f80     imageFile.obj
 0002:00000f80       $unwind$?remove@ImageFileReaderTable@@QEAAXPEAVImageFileReader@@@Z 0000000180004f80     imageFile.obj
 0002:00000f80       $unwind$JIMAGE_GetResource 0000000180004f80     jimage.obj
 0002:00000f80       $unwind$JIMAGE_PackageToModule 0000000180004f80     jimage.obj
 0002:00000f80       $unwind$??0SimpleCriticalSection@@QEAA@XZ 0000000180004f80     osSupport_windows.obj
 0002:00000f80       $unwind$__raise_securityfailure 0000000180004f80     MSVCRT:gs_report.obj
 0002:00000f80       $unwind$??2@YAPEAX_K@Z     0000000180004f80     MSVCRT:new_scalar.obj
 0002:00000f80       $unwind$??_Gtype_info@@UEAAPEAXI@Z 0000000180004f80     MSVCRT:std_type_info_static.obj
 0002:00000f80       $unwind$??0bad_alloc@std@@QEAA@AEBV01@@Z 0000000180004f80     MSVCRT:throw_bad_alloc.obj
 0002:00000f80       $unwind$??0bad_array_new_length@std@@QEAA@AEBV01@@Z 0000000180004f80     MSVCRT:throw_bad_alloc.obj
 0002:00000f80       $unwind$??0exception@std@@QEAA@AEBV01@@Z 0000000180004f80     MSVCRT:throw_bad_alloc.obj
 0002:00000f80       $unwind$__scrt_initialize_onexit_tables 0000000180004f80     MSVCRT:utility.obj
 0002:00000f80       $unwind$__scrt_release_startup_lock 0000000180004f80     MSVCRT:utility.obj
 0002:00000f80       $unwind$__scrt_uninitialize_crt 0000000180004f80     MSVCRT:utility.obj
 0002:00000f88       $unwind$?get_decompressor@ImageDecompressor@@SAPEAV1@PEBD@Z 0000000180004f88     imageDecompressor.obj
 0002:00000f88       $unwind$__scrt_dllmain_exception_filter 0000000180004f88     MSVCRT:utility.obj
 0002:00000f9c       $unwind$?decompress_resource@ImageDecompressor@@SAXPEAE0_KPEBVImageStrings@@PEAVEndian@@@Z 0000000180004f9c     imageDecompressor.obj
 0002:00000fb8       $unwind$?decompress_resource@ZipDecompressor@@UEAAXPEAE0PEAUResourceHeader@@PEBVImageStrings@@@Z 0000000180004fb8     imageDecompressor.obj
 0002:00000fc0       $unwind$?decompress_int@SharedStringDecompressor@@CAHAEAPEAE@Z 0000000180004fc0     imageDecompressor.obj
 0002:00000fc0       $unwind$?set_data@ImageLocation@@QEAAXPEAE@Z 0000000180004fc0     imageFile.obj
 0002:00000fc8       $unwind$?decompress_resource@SharedStringDecompressor@@UEAAXPEAE0PEAUResourceHeader@@PEBVImageStrings@@@Z 0000000180004fc8     imageDecompressor.obj
 0002:00000fe0       $unwind$?add@ImageFileReaderTable@@QEAAXPEAVImageFileReader@@@Z 0000000180004fe0     imageFile.obj
 0002:00000fe0       $unwind$?find@ImageStrings@@SAHPEAVEndian@@PEBDPEAHI@Z 0000000180004fe0     imageFile.obj
 0002:00000fe0       $unwind$?find_image@ImageFileReader@@SAPEAV1@PEBD@Z 0000000180004fe0     imageFile.obj
 0002:00000fe0       $unwind$?find_location@ImageFileReader@@QEBA_NPEBDAEAVImageLocation@@@Z 0000000180004fe0     imageFile.obj
 0002:00000fe0       $unwind$?open@ImageFileReader@@QEAA_NXZ 0000000180004fe0     imageFile.obj
 0002:00000fe0       $unwind$?verify_location@ImageFileReader@@QEBA_NAEAVImageLocation@@PEBD@Z 0000000180004fe0     imageFile.obj
 0002:00000fe0       $unwind$_DllMainCRTStartup 0000000180004fe0     MSVCRT:dll_dllmain.obj
 0002:00000ff0       $unwind$?package_to_module@ImageModuleData@@QEAAPEBDPEBD@Z 0000000180004ff0     imageFile.obj
 0002:0000100c       $unwind$?open@ImageFileReader@@SAPEAV1@PEBD_N@Z 000000018000500c     imageFile.obj
 0002:00001024       $unwind$?find_location_index@ImageFileReader@@QEBAIPEBDPEA_K@Z 0000000180005024     imageFile.obj
 0002:0000103c       $unwind$?get_resource@ImageFileReader@@QEBAXIPEAE@Z 000000018000503c     imageFile.obj
 0002:00001050       $unwind$?get_resource@ImageFileReader@@QEBAXAEAVImageLocation@@PEAE@Z 0000000180005050     imageFile.obj
 0002:00001068       $unwind$??__E?_reader_table@ImageFileReader@@0VImageFileReaderTable@@A@@YAXXZ 0000000180005068     imageFile.obj
 0002:00001068       $unwind$__scrt_initialize_default_local_stdio_options 0000000180005068     MSVCRT:default_local_stdio_options.obj
 0002:00001068       $unwind$?dllmain_crt_dispatch@@YAHQEAUHINSTANCE__@@KQEAX@Z 0000000180005068     MSVCRT:dll_dllmain.obj
 0002:00001068       $unwind$DllMain            0000000180005068     MSVCRT:dll_dllmain_stub.obj
 0002:00001068       $unwind$__report_rangecheckfailure 0000000180005068     MSVCRT:gs_report.obj
 0002:00001068       $unwind$__GSHandlerCheck   0000000180005068     MSVCRT:gshandler.obj
 0002:00001068       $unwind$__scrt_acquire_startup_lock 0000000180005068     MSVCRT:utility.obj
 0002:00001068       $unwind$__scrt_dllmain_after_initialize_c 0000000180005068     MSVCRT:utility.obj
 0002:00001068       $unwind$__scrt_dllmain_before_initialize_c 0000000180005068     MSVCRT:utility.obj
 0002:00001068       $unwind$__scrt_dllmain_crt_thread_attach 0000000180005068     MSVCRT:utility.obj
 0002:00001068       $unwind$__scrt_dllmain_crt_thread_detach 0000000180005068     MSVCRT:utility.obj
 0002:00001068       $unwind$__scrt_dllmain_uninitialize_c 0000000180005068     MSVCRT:utility.obj
 0002:00001068       $unwind$__scrt_dllmain_uninitialize_critical 0000000180005068     MSVCRT:utility.obj
 0002:00001068       $unwind$__scrt_initialize_crt 0000000180005068     MSVCRT:utility.obj
 0002:00001070       $unwind$JIMAGE_FindResource 0000000180005070     jimage.obj
 0002:00001090       $unwind$JIMAGE_ResourceIterator 0000000180005090     jimage.obj
 0002:000010b4       $unwind$?size@osSupport@@SA_JPEBD@Z 00000001800050b4     osSupport_windows.obj
 0002:000010c4       $unwind$?read@osSupport@@SA_JHPEAD_J1@Z 00000001800050c4     osSupport_windows.obj
 0002:000010d8       $unwind$?map_memory@osSupport@@SAPEAXHPEBD_K1@Z 00000001800050d8     osSupport_windows.obj
 0002:000010f0       $unwind$__GSHandlerCheckCommon 00000001800050f0     MSVCRT:gshandler.obj
 0002:000010f8       $xdatasym                  00000001800050f8     MSVCRT:amdsecgs.obj
 0002:000010fc       $unwind$__report_securityfailure 00000001800050fc     MSVCRT:gs_report.obj
 0002:00001104       $unwind$__report_gsfailure 0000000180005104     MSVCRT:gs_report.obj
 0002:0000110c       $unwind$capture_current_context 000000018000510c     MSVCRT:gs_report.obj
 0002:00001118       $unwind$capture_previous_context 0000000180005118     MSVCRT:gs_report.obj
 0002:00001128       $xdatasym                  0000000180005128     MSVCRT:chkstk.obj
 0002:00001130       $unwind$?dllmain_crt_process_attach@@YAHQEAUHINSTANCE__@@QEAX@Z 0000000180005130     MSVCRT:dll_dllmain.obj
 0002:0000116c       $unwind$?fin$0@?0??dllmain_crt_process_attach@@YAHQEAUHINSTANCE__@@QEAX@Z@4HA 000000018000516c     MSVCRT:dll_dllmain.obj
 0002:0000116c       $unwind$?fin$0@?0??dllmain_crt_process_detach@@YAH_N@Z@4HA 000000018000516c     MSVCRT:dll_dllmain.obj
 0002:0000116c       $unwind$?fin$1@?0??dllmain_crt_process_detach@@YAH_N@Z@4HA 000000018000516c     MSVCRT:dll_dllmain.obj
 0002:00001174       $unwind$?dllmain_crt_process_detach@@YAH_N@Z 0000000180005174     MSVCRT:dll_dllmain.obj
 0002:000011c8       $unwind$?dllmain_dispatch@@YAHQEAUHINSTANCE__@@KQEAX@Z 00000001800051c8     MSVCRT:dll_dllmain.obj
 0002:000011f0       $unwind$?filt$0@?0??dllmain_dispatch@@YAHQEAUHINSTANCE__@@KQEAX@Z@4HA 00000001800051f0     MSVCRT:dll_dllmain.obj
 0002:000011f8       $unwind$_RTC_Initialize    00000001800051f8     MSVCRT:initsect.obj
 0002:000011f8       $unwind$_RTC_Terminate     00000001800051f8     MSVCRT:initsect.obj
 0002:000011f8       $unwind$??_Gbad_alloc@std@@UEAAPEAXI@Z 00000001800051f8     MSVCRT:throw_bad_alloc.obj
 0002:000011f8       $unwind$??_Gbad_array_new_length@std@@UEAAPEAXI@Z 00000001800051f8     MSVCRT:throw_bad_alloc.obj
 0002:000011f8       $unwind$??_Gexception@std@@UEAAPEAXI@Z 00000001800051f8     MSVCRT:throw_bad_alloc.obj
 0002:00001204       $unwind$?__scrt_throw_std_bad_alloc@@YAXXZ 0000000180005204     MSVCRT:throw_bad_alloc.obj
 0002:00001204       $unwind$?__scrt_throw_std_bad_array_new_length@@YAXXZ 0000000180005204     MSVCRT:throw_bad_alloc.obj
 0002:0000120c       $unwind$__security_init_cookie 000000018000520c     MSVCRT:gs_support.obj
 0002:00001218       $unwind$__scrt_is_nonwritable_in_current_image 0000000180005218     MSVCRT:utility.obj
 0002:00001238       $unwind$__scrt_is_nonwritable_in_current_image$filt$0 0000000180005238     MSVCRT:utility.obj
 0002:00001240       $unwind$__scrt_fastfail    0000000180005240     MSVCRT:utility_desktop.obj
 0002:00001250       $unwind$__isa_available_init 0000000180005250     MSVCRT:cpu_disp.obj
 0002:00001268       $xdatasym                  0000000180005268     MSVCRT:guard_dispatch.obj
 0002:00001270       $xdatasym                  0000000180005270     MSVCRT:guard_xfg_dispatch.obj
 0002:00001370       .edata                     0000000180005370     jimage.exp
 0002:00001398       rgpv                       0000000180005398     jimage.exp
 0002:000013b4       rgszName                   00000001800053b4     jimage.exp
 0002:000013d0       rgwOrd                     00000001800053d0     jimage.exp
 0002:000013de       szName                     00000001800053de     jimage.exp
 0002:000013e9       $N00001                    00000001800053e9     jimage.exp
 0002:000013f6       $N00002                    00000001800053f6     jimage.exp
 0002:0000140a       $N00003                    000000018000540a     jimage.exp
 0002:0000141d       $N00004                    000000018000541d     jimage.exp
 0002:00001429       $N00005                    0000000180005429     jimage.exp
 0002:00001440       $N00006                    0000000180005440     jimage.exp
 0002:00001458       $N00007                    0000000180005458     jimage.exp
 0002:00001766       .idata$6                   0000000180005766     jvm:jvm.dll
 0002:00001994       .idata$6                   0000000180005994     kernel32:KERNEL32.dll
 0002:00001a36       .idata$6                   0000000180005a36     vcruntime:VCRUNTIME140.dll
 0002:00001bb0       .idata$6                   0000000180005bb0     ucrt:api-ms-win-crt-stdio-l1-1-0.dll
 0002:00001bd0       .idata$6                   0000000180005bd0     ucrt:api-ms-win-crt-string-l1-1-0.dll
 0002:00001bf2       .idata$6                   0000000180005bf2     ucrt:api-ms-win-crt-heap-l1-1-0.dll
 0002:00001c12       .idata$6                   0000000180005c12     ucrt:api-ms-win-crt-filesystem-l1-1-0.dll
 0002:00001c38       .idata$6                   0000000180005c38     ucrt:api-ms-win-crt-runtime-l1-1-0.dll
 0003:00000270       ?ZipInflateFully@@3P6AEPEAX_J01PEAPEAD@ZEA 0000000180006270     imageDecompressor.obj
 0003:000002b0       GS_ExceptionRecord         00000001800062b0     MSVCRT:gs_report.obj
 0003:00000350       GS_ContextRecord           0000000180006350     MSVCRT:gs_report.obj
 0003:00000820       ?__proc_attached@@3HA      0000000180006820     MSVCRT:dll_dllmain.obj
 0003:00000858       ?is_initialized_as_dll@@3_NA 0000000180006858     MSVCRT:utility.obj
 0003:00000859       ?module_local_atexit_table_initialized@@3_NA 0000000180006859     MSVCRT:utility.obj
 0003:00000860       ?module_local_atexit_table@@3U_onexit_table_t@@A 0000000180006860     MSVCRT:utility.obj
 0003:00000878       ?module_local_at_quick_exit_table@@3U_onexit_table_t@@A 0000000180006878     MSVCRT:utility.obj
 0005:00000060       $R000000                   0000000180008060     jimage.dll.res
